:020000040800F2
:10000000500800208D010008751B00083D190008EC
:1000100000000000000000000000000000000000E0
:10002000000000000000000000000000791B000834
:100030000000000000000000771B00087B1B000888
:100040009F010008000000009F0100089F010008B8
:100050009F0100089F0100089F0100089F01000800
:10006000000000009F010008AD050008BD05000864
:100070009F0100089F0100089F0100080000000088
:100080009F01000800000000000000009F01000820
:10009000000000009F0100089F0100089F01000868
:1000A000000000009F010008000000002522000859
:1000B00000F002F800F03EF80CA030C80838241810
:1000C0002D18A246671EAB4654465D46AC4201D190
:1000D00000F030F87E460F3E0FCCB6460126334284
:1000E00000D0FB1AA246AB46334318474426000013
:1000F00064260000103A02D378C878C1FAD85207B3
:1001000001D330C830C101D504680C6070470000CD
:100110000023002400250026103A01D378C1FBD823
:10012000520700D330C100D50B6070471FB51FBD0B
:1001300010B510BD00F0E9F91146FFF7F7FF02F026
:10014000F9F800F001FA03B4FFF7F2FF03BC00F086
:1001500007FA000070B505460C46164602E00FCCC3
:100160000FC5103E102EFAD2082E02D303CC03C5C1
:10017000083E042E07D301CC01C5361F03E02178C9
:100180002970641C6D1C761EF9D270BD074880472B
:1001900007480047FEE7FEE7FEE7FEE7FEE7FEE76B
:1001A00004480549054A064B704700006D1C0008CD
:1001B000B100000850020020500800205004002028
:1001C0005004002010B5202A04DB0846203AD04015
:1001D000002110BD0B462024D340D040A21A9140EC
:1001E0000843194610BDFEB5054610460C46184397
:1001F00073D0AE468C460020AD1A01469C4167D3B1
:100200006646002701243D46B61A9D4102D3134697
:100210003A462124654676462F04360C3E432D0C83
:10022000B61A9D4104D3150C1B042B431204103441
:10023000654676462F06360A3E432D0AB61A9D417C
:1002400004D3150E1B022B43120208346546764672
:100250002F0736093E432D09B61A9D4104D3150FC9
:100260001B012B431201241D65467646AF07B608D5
:100270003E43AD08B61A9D4104D3950F9B002B4316
:100280009200A41C65467646EF0776083E436D084B
:10029000B61A9D411AD392185B41641C16E00018EF
:1002A000764665464941B71A9D410191009009D3B0
:1002B0006046B11A98418E468446009801990025FF
:1002C000401C6941DD0752082A435B08641EE6D5DD
:1002D0007246634603B0F0BDFFE700200146C0460A
:1002E000C0462A462346F5E7F8B5042A2CD38307EF
:1002F00012D00B78491C0370401C521E83070BD090
:100300000B78491C0370401C521E830704D00B78E5
:10031000491C0370401C521E8B079B0F05D0C91A45
:10032000DF002023DE1B08C90AE0FFF713FFF8BD3A
:100330001D4608C9FD401C46B4402C4310C0121F86
:10034000042AF5D2F308C91A521EF0D40B78491CBE
:100350000370401C521EEAD40B78491C0370401CE9
:10036000012AE4D409780170F8BD01E004C0091F36
:100370000429FBD28B0701D50280801CC90700D05D
:100380000270704700290BD0C30702D00270401CD6
:10039000491E022904D3830702D50280801C891ECE
:1003A000E3E70022EEE70022DFE7002203098B42A9
:1003B0002CD3030A8B4211D300239C464EE0034604
:1003C0000B433CD4002243088B4231D303098B42B8
:1003D0001CD3030A8B4201D394463FE0C3098B42EE
:1003E00001D3CB01C01A524183098B4201D38B0147
:1003F000C01A524143098B4201D34B01C01A5241EA
:1004000003098B4201D30B01C01A5241C3088B422E
:1004100001D3CB00C01A524183088B4201D38B0019
:10042000C01A524143088B4201D34B00C01A5241BB
:10043000411A00D201465241104670475DE0CA0F92
:1004400000D04942031000D34042534000229C4652
:1004500003098B422DD3030A8B4212D3FC2289015C
:1004600012BA030A8B420CD3890192118B4208D332
:10047000890192118B4204D389013AD0921100E094
:100480008909C3098B4201D3CB01C01A52418309A8
:100490008B4201D38B01C01A524143098B4201D3D5
:1004A0004B01C01A524103098B4201D30B01C01A00
:1004B0005241C3088B4201D3CB00C01A524183087A
:1004C0008B4201D38B00C01A5241D9D243088B42D0
:1004D00001D34B00C01A5241411A00D20146634673
:1004E00052415B10104601D34042002B00D54942D7
:1004F000704763465B1000D3404201B50020C04600
:10050000C04602BD704770477047754600F024F83A
:10051000AE46050069465346C008C000854618B07F
:1005200020B5FFF73DFE60BC00274908B64600260F
:10053000C0C5C0C5C0C5C0C5C0C5C0C5C0C5C0C593
:10054000403D49008D46704710B50446C046C04640
:100550002046FFF7F8FD10BD00487047F00100206D
:1005600001491820ABBEFEE7260002007047417823
:1005700002780802104340BA7047000070B50A4D77
:10058000FF22EE1D1346F93605E0047854402A5D3B
:100590005A40335D401C0C46491E89B2002CF4D1F0
:1005A0001002184370BD00001825000810B502485D
:1005B00000F0F5F810BD00004801002010B5024819
:1005C00000F0EDF810BD00008C01002010B50446CD
:1005D0000068054940181421FFF7E7FE80002064F9
:1005E0000248E06310BD0000F8FFFDBF00000240BC
:1005F00030B5056C0124AC40C56B6C600468636069
:100600004368102B036803D099600068C26030BD56
:100610009A600068C16030BD72B6FEE706490020EE
:10062000C861064801690422114301610169402241
:100630001143016170470000D001002000200240FA
:10064000064A0021D16106490A6902231A430A6158
:10065000486108694022104308617047D0010020BA
:100660000020024010B5054B0022DA61044A1369EC
:10067000012423431361018010BD0000D00100203C
:100680000020024010B50B4A0020D168CB060A4971
:1006900004D5C86902231843C8611020D3685B07DA
:1006A00005D5CB6901242343CB6104210843D060E5
:1006B00010BD000000200240D001002070B50446AB
:1006C00000F088FA0546104E0AE0601C08D0002CA5
:1006D00004D000F07FFA401BA04201D9032070BD76
:1006E000F068C007F1D1F068800601D52020F060E5
:1006F000F068C00602D4F068400703D5FFF7C2FFD8
:10070000012070BD002070BD0020024030B50146C0
:1007100020314A780023022A04D0042282630B701D
:10072000012030BD026814680E25AC4314600268D5
:1007300014686408640014600125046C2A46C06BC8
:10074000A24042604D700B70002030BD70B5002497
:10075000014620314A78022A03D004218163012412
:1007600016E0026813680E25AB4313600268136835
:100770005B085B0013600125036C2A469A40C36B3B
:100780005A604D7000220A70416B002900D08847E2
:10079000204670BD806B7047203040787047F0B4C1
:1007A000C16B0C6801680B680422056C1646AE40EC
:1007B00026420DD05E070BD50B689B0602D40B6852
:1007C00093430B60016C8A40C16B4A60C16A19E0B7
:1007D0000227AF400246274001262032002F15D0C5
:1007E0009F0713D50B689B0604D40B680A24A34308
:1007F0000B605670036C02219940C36B5960002155
:100800001170816A002916D0F0BC08470827AF4054
:10081000274210D01B070ED50B680E24A3430B6094
:10082000036C31469940C36B596086635670002152
:100830001170016BE6E7F0BC7047000070B5040072
:100840001FD00220254620356870206802680E49B6
:10085000A3680A40616826691943E3683343194372
:1008600063691943A3691943E3691943114301609B
:100870002046FFF7ABFE0020A063012169702870BD
:1008800070BD012070BD00000FC0FFFFF8B5044629
:100890008C46203001780025012909D001260670F8
:1008A00047780021012F05D0017002252846F8BDA8
:1008B0000220F8BD02274770A1632068016849083B
:1008C0004900016061462046FFF792FEE06A002879
:1008D0002068016802D00E22114306E00A2211436B
:1008E000016020680168042291430160206801686A
:1008F00031430160DAE7000070B5044600F06AF9A0
:100900000546601C02D004480078241800F062F903
:10091000401BA042FAD370BD14000020F8B5054674
:1009200023480F46017E012601290BD001210176C3
:100930002868204C012807D02046FFF7BFFE00287A
:1009400013D030E00220F8BD2046FFF7B7FE0028A4
:1009500029D1FFF763FE2046FFF7B0FE0646164892
:1009600001690422914301611DE00020C043386009
:100970006C6812E02046FFF763FE0E48FFF79EFE0C
:1009800006460D480169022291430161002E01D003
:100990003C6008E0012080022418A8686968800291
:1009A0004018A042E6D80248002101763046F8BD42
:1009B000D001002050C3000000200240034801691C
:1009C0008022114301610020704700000020024096
:1009D000F0B51FB405461A480024017E16461F468E
:1009E000012907D0012101761648FFF767FE00288C
:1009F00003D021E0022005B0F0BD012D1AD0022D58
:100A000018D0042516E0220130463946FFF7DAFBFC
:100A100081B2019862001018FFF724FE0948FFF721
:100A20004DFE09490A69520852000A61002803D1A3
:100A3000641CE4B2AC42E6D3014900220A76DAE74C
:100A4000D001002050C300000020024006490020D1
:100A50000A69120607D5054A4A60054A4A600969CB
:100A6000090600D501207047002002402301674598
:100A7000AB89EFCDF8B5002294E0012797403B40C9
:100A80007ED00C79A407A40F012C01D0022C10D128
:100A9000856854000326A640B543CE68A6402E4381
:100AA000866044680D79BC43ED06ED0F9540254303
:100AB00045600C79E443A40708D0C56854000326B8
:100AC000A640B5438E68A6402E43C6600C79A407A5
:100AD000A40F022C0CD1D408A40027183D6A540797
:100AE000E40E0F26A640B5430E69A6402E433E6293
:100AF000056854000326A640B5430E79B607B60F25
:100B0000A6402E4306604C68A403A40F49D0284C8D
:100B1000A56901263543A561A46995083440009470
:100B2000244CAD002F19BD689407240F0F26A64052
:100B3000B5430926F606B04201D100260FE01E4E4D
:100B4000B04201D101260AE01C4EB04201D102267A
:100B500005E01B4EB04201D1032600E00526A64069
:100B60002E43BE60174D2C684E689C43F60300D59B
:100B70001C432C606C684E689C43B60302D500E0B1
:100B80000FE01C436C60AC684E689C43F60200D5D5
:100B90001C43AC60EC684E689C43B60200D51C4315
:100BA000EC60521C0B681C46D44000D065E7F8BDD1
:100BB0000010024000000140000400480008004806
:100BC000000C004800040140002A01D081617047F8
:100BD000816270470148806870470000140000205F
:100BE00070B504000FD021681548086021681548C9
:100BF000086003CC41602068083C21688860FFF7EA
:100C0000E9FF05460CE0012070BDFFF7E3FF401B44
:100C1000272805D92068C068400701D0032070BD8F
:100C20002068C0684007F0D120680269E1688A4204
:100C300001D0016101E004490160002070BD0000A5
:100C4000CCCC000055550000AAAA0000006802495B
:100C50000160002070470000AAAA000002488168D5
:100C600002788918816070471400002010B506488A
:100C70000168102211430160032000F007F800F022
:100C800027F8002010BD00000020024070B5044687
:100C90000D4D7D202978C000FFF787FB01460B48EA
:100CA0000068FFF782FB00F055FB002809D1042CF7
:100CB00007D200222146401E00F02AF800206C6076
:100CC00070BD012070BD0000140000202000002035
:100CD00008B5084881690122114381618169114089
:100CE0000091C26901040A43C261C06908400090D2
:100CF00008BD000000100240002805DBC106C90E37
:100D000001208840014908607047000000E100E0D0
:100D100010B501F0EDFA10BDF8B504460068364D87
:100D2000C00354D5E8690026C00007D4E869290447
:100D30000843E861E8690840012600902F480168EF
:100D4000C90511D4014608688A1510430860FFF7E9
:100D500041FF074604E0FFF73DFFC01B642823D88E
:100D600026480068C005F6D5286A03210902084014
:100D70001FD062680A4082421BD0286A2A6A8843D0
:100D8000012109040A432A622A6A8A432A622862E4
:100D9000C0070ED0FFF71EFF074607E0FFF71AFF58
:100DA000C11B1748814201D90320F8BD286A80077A
:100DB000F4D5286A03210902884361680843286240
:100DC000002E04D0E869012109078843E8612078F2
:100DD000C00705D0286BA1688008800008432863FD
:100DE0002078800605D5286B10218843E1680843E8
:100DF00028630020F8BD0000001002400070004091
:100E000088130000F8B50D4604005AD03A4800682F
:100E1000C007C00FA8420AD23748016849084900F4
:100E2000294301600068C007C00FA84249D120686B
:100E3000324E81070CD5400704D57068072109029E
:100E4000084370607068F0218843A16808437060AF
:100E50002078C00725D0606801280ED031680228AC
:100E60000ED0890700292CDA7168890889000143AE
:100E70007160FFF7AFFE07460CE031688903F1E7C8
:100E80008901EFE7FFF7A6FEC11B1D48814201D98A
:100E90000320F8BD70680C21084061688900884211
:100EA000F0D115480168C907C90FA9420BD90168DB
:100EB00049084900294301600068C007C00FA842E3
:100EC00001D00120F8BD2078400706D570680721C1
:100ED00009028843E1680843706000F027F87168F0
:100EE000084A0906090F515CC840074908600320F9
:100EF000FFF7CCFE0020F8BD0020024000100240A9
:100F00008813000018270008200000200448054925
:100F100000684968044A4905490F515CC840704758
:100F200020000020001002402827000810B514A05F
:100F30000FC888B06C460FC415A00FC80FC4184A5C
:100F400053680C20194601401648042916D0082978
:100F500014D19902090F6C46645CD16A04AA09078E
:100F6000090F525CD90305D500231946FFF73BF959
:100F7000214601E020460C4901F0A2F908B010BD5D
:100F800002030405060708090A0B0C0D0E0F1010CA
:100F90000102030405060708090A0B0C0D0E0F10C9
:100FA0000010024000127A0000093D00FEB5040066
:100FB00076D02078E44DC00753D068680007800FD2
:100FC000012807D068680007800F022809D16868E7
:100FD000C00306D52868800343D560680028E7D0A1
:100FE0003FE06068012813D001218904002814D053
:100FF000052818D02A68881082432A602868884308
:1010000028606068002820D0FFF7E4FD064618E05D
:101010002868012109040843F2E728680122120424
:1010200090432860EAE7286808432860296801207F
:10103000000401432960E4E7FFF7CCFD801B64282E
:1010400075D828688003F7D50BE0FFF7C3FD064687
:1010500004E0FFF7BFFD801B6428F1D828688003F7
:10106000F7D4207801268007002843DA6868000753
:10107000800F07D068680007800F022811D16868C8
:10108000C0030ED42868800702D5E068012807D184
:101090002868F82188432169C9000843286029E0AD
:1010A0004DE1E0680028286815D030432860FFF73C
:1010B00091FD074604E0FFF78DFDC01B0228BFD855
:1010C00028688007F7D52968F82081432069C00087
:1010D000014329600EE0400840002860FFF77AFDD8
:1010E000074604E0FFF776FDC01B0228A8D8286851
:1010F0008007F7D42078000722D5E0690028686AC5
:101100000ED030436862FFF765FD074604E0FFF745
:1011100061FDC01B022893D8686A8007F7D50FE0ED
:10112000400840006862FFF755FD074605E09DE076
:10113000FFF750FDC01B02288FD8686A8007F7D4DC
:10114000207804274007002860DA00200190E86931
:10115000C00008D4E969B8060143E961E9690140C2
:1011600001200091019079480168C90511D40168F6
:10117000821511430160FFF72DFD009005E0FFF798
:1011800029FD0099401A642870D870480068C0058D
:10119000F5D5A06801280AD0002801D0052810D074
:1011A000286A400840002862286AB84301E0286A9B
:1011B00030432862A068002812D0FFF70BFD009092
:1011C0000AE0286A38432862F1E7FFF703FD009937
:1011D000411A5F48814249D8286A8007F5D50DE059
:1011E000FFF7F8FC009006E0FFF7F4FC0099411AC5
:1011F000574881423AD8286A8007F5D401980028D8
:1012000004D0E869012109078843E8612078C00615
:1012100035D5606901280CD0401D686B23D0384358
:101220006863686B400840006863FFF7D3FC0646BC
:1012300022E0686B38436863686B30436863FFF78C
:10124000C9FC064604E0FFF7C5FC801B02285BD8FA
:10125000686B8007F7D5686BF8218843A169C900DE
:10126000084368630BE0B8436863F4E74CE0FFF7BA
:10127000B1FC801B022847D8686B8007F7D4206A2E
:1012800000285ED069680907890F022942D001272A
:101290003F060228286805D0B8432860FFF79AFC6B
:1012A000044633E0B8432860FFF794FC064604E0A8
:1012B000FFF790FC801B022826D828688001F7D40D
:1012C000E86AE16A000900010843E862616AA06A0D
:1012D000084369683D221204914308436860286806
:1012E00038432860FFF776FC044604E0FFF772FC01
:1012F000001B022808D828688001F7D521E0FFF7F5
:1013000069FC001B022801D90320FEBD286880016A
:10131000F5D416E00128F8D06868E96A01221204C1
:10132000636A02409A420AD10907E26A090F9142B0
:1013300005D10F2189040840A16A884201D001200B
:10134000FEBD0020FEBD0000001002400070004005
:1013500088130000094910B5401E884201D90120B8
:1013600010BD074C60610321081F00F0C1FF002081
:10137000A06107202061002010BD0000FFFFFF00DA
:1013800000E000E07047F8B5816F0446C66F006862
:1013900082682546120610278035002A1BDA21298B
:1013A00019D1EFF31081012282F310888268802323
:1013B0009A43826081F31088E06E002808D0FFF71E
:1013C000A5F9002804D0E06EFFF7E4F9202824D026
:1013D000204600F0C2FD2068816849061BD5222EF8
:1013E00019D1EFF31081012282F310888268402323
:1013F0009A43826081F31088206F002808D0FFF79D
:1014000085F9002804D0206FFFF7C4F9202804D004
:10141000204600F074FD0020F8BD2F600320F8BDC9
:1014200070470000F8B502680446D06911689668F4
:101430009C4B05461D402023002D75D0F7079A4D83
:10144000FF0FBC460D402F436DD02546C7078035A2
:10145000002F06D0CF0504D5012717622A683A432A
:101460002A60820708D5F20706D0276802223A626E
:101470002A6804273A432A60420708D5F20706D0B3
:101480002668042232622A68022632432A60020752
:101490000AD50A461A406646324305D02668082215
:1014A00032622E6816432E60020508D54A0106D521
:1014B00001222668D20232622A681A432A602A6808
:1014C000002A39D0800606D5880604D5616E002929
:1014D00001D020468847286821688968490602D4D7
:1014E000282108422DD0204600F009FD206881689F
:1014F000490622D5EFF31081012282F31088836818
:1015000040229343836081F31088206F002814D019
:1015100066494163206FFFF719F900280CD0206F4E
:10152000416B08E000E012E0850610D58D060ED56F
:10153000616E9DE020468847F8BD2046FFF770FFAA
:10154000F8BD2046FFF76CFF00202860F8BD256E2F
:10155000012D7DD1C5067BD5CD0679D51026166225
:1015600020688168254649064035002945DA226F02
:10157000116849680904090CE8D02F8B8F42E5D91E
:1015800069839169202933D0EFF31081012282F31E
:10159000108802683701BA43026081F31088EFF3C4
:1015A0001081012080F31088206882685208520060
:1015B000826081F31088EFF31081012080F310889E
:1015C000206882684027BA43826081F31088E3670D
:1015D00000202066EFF31081012080F3108820683E
:1015E0000268B243026081F31088206FFFF78EF823
:1015F000288B698B401A81B231E0298B6A8B891A5A
:101600006A8B89B2002AA1D000299FD0EFF3108203
:10161000012585F310880568FF272137BD43056044
:1016200082F31088EFF31082012080F31088206885
:1016300085686D086D00856082F31088E36700207F
:101640002066EFF310826066012080F3108800E0CE
:1016500009E020680368B343036082F310882046E2
:10166000FFF790FEF8BD050606D50D0604D5A16E60
:10167000002900D05EE7F8BD4006FCD54806FAD543
:101680002046EFF31081012484F31088146840256C
:10169000AC43146081F3108883670021816600F0F9
:1016A0004BF9F8BD0F080000200100049D1D000843
:1016B00010B5040003D0A06F002802D007E001207D
:1016C00010BD002174200155204600F027F8242089
:1016D000A06720680168490849000160204600F0C1
:1016E0004DFC0128ECD0606A002802D0204600F0B2
:1016F000BEFA206841680122D2029143416020680D
:1017000081680822914381602068016801221143A9
:101710000160204600F010FB10BD0000F0B587B05E
:10172000044614216846FEF73EFE3449206888428C
:1017300061D133488269012189030A438261826948
:101740000A4005924269C9000A4342614069002685
:1017500008400590032040020090022001900320E1
:10176000039001200490092002966946C006FFF705
:1017700081F92448244D802741C52E60AE60EE607B
:101780006F6080142E6168611F48083DFFF756F8AE
:10179000002801D0FEF740FF25676C621A4D1948FA
:1017A0004435143028601020291DC1C12E616E619E
:1017B0000002AE61E8612846FFF740F8002801D03A
:1017C000FEF72AFF11480168421511430160E566E2
:1017D000002211461B206C62FFF79AFA1B20FFF7CC
:1017E0008BFA094A843A1068016810231943016092
:1017F00011685020086207B0F0BD000000380140B9
:10180000001002403000024048010020000001406A
:1018100070B5C36F202B2BD100290BD0002A09D023
:10182000012483682403A34206D10369002B03D15A
:10183000CB0701D0012070BD034660331C7D012C15
:1018400016D001241C750023036603685C6824021B
:101850000BD5EFF31084012585F310881D68012650
:10186000B60635431D6084F3108800F015FC70BD8A
:10187000022070BD70477047F8B50446806F20287D
:1018800052D100290BD0002A09D00123A0681B03E4
:10189000984206D12069002803D1C80701D0012051
:1018A000F8BD25466035287D01283DD001202875EA
:1018B00020464030E164028242820026274680377B
:1018C0003E602120A067E06E00281BD0174981628E
:1018D000E16E1748C862E16E16480863E06E134671
:1018E0004663E06C216884460A4628326146E06E11
:1018F000FEF7CCFF002805D0102038602E75202080
:10190000A067CCE72168402008622E75EFF31081B4
:10191000012080F310882068826880231A43826047
:1019200081F310880020F8BD0220F8BDAB1E00082E
:10193000F51E0008B11D000870477047FEE7000063
:10194000F8B5384D281DFEF712FE04B2A81CFEF7AC
:101950000EFE064606212846FEF710FE024600202F
:101960002F46203F295C3954401CC0B20628F9D3C9
:10197000110AD0B2B9712C4AF8710F2E06D0FF238C
:10198000F533042E2BD0052E33D045E0AB799942A8
:1019900042D1E97988423FD1601EF6280ED8D48022
:1019A000012080F3108800F081FD002831D12878D3
:1019B00000282ED0082000F059FD2AE0FF203871C1
:1019C000787106211748FEF7D9FD010AB971F8713F
:1019D0002878002820D0082000F048FD1CE0AE79CF
:1019E000B14219D1E979884216D19C4214DB548066
:1019F00008E0AE79B1420FD1E97988420CD19C421E
:101A00000ADB9480012080F3108800F04FFD00284D
:101A1000D0D0002080F3108820210248FEF7C1FCBE
:101A2000F8BD0000640000200000002008B50C484C
:101A30004169012211434161406901211040009038
:101A400000220A20FFF764F90A20FFF755F9002267
:101A500001210B20FFF75CF90B20FFF74DF908BDC2
:101A600000100240F0B587B014216846FEF79BFCD9
:101A700023484269012189050A43426142690A40BB
:101A80000592426949110A43426142690A4005923E
:101A9000426949000A434261406909260840F60646
:101AA00005900022E8213046FFF78EF80122102130
:101AB0003046FFF789F8134F002202213846FFF71E
:101AC00083F8C82001240225694631C10320039010
:101AD00069463046FEF7CEFF30200090002002908D
:101AE0000194694603943046FEF7C4FF01940294C2
:101AF0006946384600950394FEF7BCFF07B0F0BD79
:101B0000001002400004004810B509480749016070
:101B1000062141600749C16007498160FFF760F80D
:101B2000002801D0FEF778FD10BD00000030004015
:101B3000B4000020FF0F0000B80B000010B50C48E7
:101B40000A4901604B21C901416000218160C160E7
:101B500001618161C1610C22016242614162FFF752
:101B6000A7FD002801D0FEF757FD10BD0038014049
:101B7000C4000020FEE77047704710B500F004F87D
:101B8000FFF76CF810BD000030B5184B5868012401
:101B9000002804D05868401E586000D11C70144DB5
:101BA00000210C20484340194268002A09D04268AD
:101BB000521E426005D144700278012A01D1826828
:101BC0004260491CC9B20429EBD39868401C986054
:101BD0009868084A0021904200D199605878401CCA
:101BE000C0B258700A2800D3597030BD08000020D8
:101BF00084000020FFFFFF7F70B594B0302168465D
:101C0000FEF7D1FB00240F94092002250E940090CA
:101C10001394E803012609900C940D94109400018C
:101C20001194129401960A90079608950B946846B1
:101C3000FFF7BCF9002801D072B6FEE707200C9030
:101C40000E9401210D950F940CA8FFF7DBF80028E6
:101C500001D072B6FEE710A810961294FFF75CF858
:101C6000002801D072B6FEE714B070BD704710B501
:101C7000818CC90707D001684A6801235B049A4335
:101C8000836A1A434A60818C890707D501684A68CC
:101C900001231B049A43C36A1A434A60818C490793
:101CA00007D501684A6801239B049A43036B1A43D2
:101CB0004A60818C090707D501684A680123DB0364
:101CC0009A43436B1A434A60818CC90607D5016861
:101CD0008A6801231B039A43836B1A438A60818CB1
:101CE000890607D501688A6801235B039A43C36BA1
:101CF0001A438A60818C490612D501684B6801221B
:101D00001205046C934323434B60016C914207D14D
:101D100001684A6803235B059A43436C1A434A608F
:101D2000818C090607D501684A680123DB04806CB1
:101D30009A4302434A6010BDF8B50446002580303E
:101D40000560FEF747FF074620680068124E00074F
:101D500009D501213B46002249052046009600F0A6
:101D6000F5F900280DD12068006840070BD5012146
:101D70003B46002289052046009600F0E7F900283E
:101D800001D00320F8BD2020A067E06725666034FD
:101D900025750020F8BD0000FFFFFF0110B5406A67
:101DA0000022014640314A834A82FFF739FB10BDC9
:101DB00070B5446AA06FE56F21688968002609063E
:101DC000002906DA212804D152200653204600F0CB
:101DD000C4F820688068400606D5222D04D15A2018
:101DE0000653204600F08BF8204680300168102210
:101DF000114301602046FFF713FB70BD10B501468B
:101E00008969406A202937D000225A210A52EFF30B
:101E10001082012181F3108801680B68FF240134CE
:101E2000A3430B6082F31088EFF31082012181F34A
:101E3000108801688B685B085B008B6082F31088F8
:101E4000EFF31082012181F3108801688B68402430
:101E5000A3438B6082F310882021C167016E0129A2
:101E60000AD1EFF3108281F3108801680B68102407
:101E7000A3430B6082F31088016E012902D0FFF7A3
:101E8000F9FC10BD5821095AFFF77CFA10BD10B5B6
:101E9000406A016E012902D0FFF7EDFC10BD582108
:101EA000095A4908FFF76EFA10BD10B50146896955
:101EB000406A20291BD0002252210A52EFF31082DF
:101EC000012181F3108801688B688024A3438B6013
:101ED00082F31088EFF31081012282F310880068EA
:101EE000026840231A43026081F3108810BDFFF797
:101EF00023FD10BD10B5406AFFF71FFD10BD10B5E2
:101F0000EFF31082012181F3108801680B68FF2430
:101F10002134A3430B6082F31088EFF31082012178
:101F200081F3108801688B685B085B008B6082F32B
:101F30001088016E01290AD1EFF3108281F3108815
:101F400001680B681024A3430B6082F310882021E2
:101F5000C16700210166416610BD10B5EFF3108224
:101F6000012181F3108801680B68C024A3430B6032
:101F700082F310882021816710BD000070B50446EF
:101F800081680069E26901436069002510430143EB
:101F9000206802683C4B1A400A430260206841688E
:101FA000032212039143E26811434160216AA06950
:101FB0000143206882680B231B029A430A43826014
:101FC0003248006B8007800F06D0012816D0022807
:101FD00016D0032810D010200122E369D2032C4927
:101FE0002C4E93422BD100280CD002280DD004286F
:101FF0000DD008283FD10EE00220EDE70420EBE7EA
:102000000820E9E7FEF782FF03E00A4603E0FEF757
:102010008DFF020033D0616850004A088018FEF737
:10202000C4F980B201461039B14224D81949491C7B
:1020300001400007420F20680A43C2601FE00028E9
:1020400006D0022807D0042807D0082813D108E0BA
:10205000FEF75CFF03E00A4603E0FEF767FF0200BD
:102060000DD0616848088018FEF79FF980B20146DC
:102070001039B14201D9012501E02168C860002072
:102080006066A066284670BDF369FFFF001002403D
:1020900000127A00EFFF0000F8B5044641654030B9
:1020A00000262746028380373E602220E0672546CF
:1020B000206F603500281BD021498162216F2148A3
:1020C000C862216F20480863206F13464663606D25
:1020D0002168844662462431206FFEF7D7FB002832
:1020E00006D0102038602E752020E0670120F8BD52
:1020F0002E75EFF31081012080F3108820680268AC
:10210000FF2301331A43026081F31088EFF310813B
:10211000012080F3108820688368012213438360C4
:1021200081F31088EFF3108182F3108820688268B1
:1021300040231A43826081F310880020F8BD00001C
:10214000FD1D00088F1E0008B11D0008FFB581B0FD
:1021500006460F46044660360A9D55E0681C53D07B
:10216000FEF738FD0499401AA84230D8002D2ED031
:1021700020680168490747D5C069C043000543D4BA
:1021800001202168C0020862EFF31081012080F372
:10219000108820680268FF23A1339A43026081F30C
:1021A0001088EFF31081012080F310882068826886
:1021B00052085200826081F310882020A067E067F7
:1021C0008034206000203075032005B0F0BDEFF3AF
:1021D0001081012080F3108820680368FF22A1325B
:1021E0009343036081F31088EFF31081012080F3A3
:1021F00010882068826852085200826081F310883B
:102200002020A067E067DDE72068C1693846884381
:1022100005D0002003998842A0D00020D5E70120F6
:10222000F8E7000010B51148FFF7FCF80F48006808
:10223000C169C943C90618D4102101620B48FFF7D0
:10224000A2F80B48017800290AD10A4909684968AF
:102250002022511ACAB2027007490848FEF744F812
:10226000202205490148FFF7D3FA10BDC400002021
:10227000000000204801002024000020640000200D
:1022800010B50D480D4C02784178E388204600785F
:102290009A4201D1082802D0002A03D008E003297D
:1022A00002D105E0082803D1062901D1FFF748FB38
:1022B0000020207010BD00006400002000000020FD
:1022C000F8B5040C8BB2264682B25E430D0C104664
:1022D000370C5843360480190021794116466E4365
:1022E000370C36048019794126466E438919F8BDAA
:1022F0008307FF22DB0E9A408907090E99400028C8
:1023000008DB830809489B001818036893430B43B4
:10231000036070470007000F0838830804489B00DB
:102320001818C36993430B43C361704700E400E08E
:1023300000ED00E0FEF79AFCFFF75EFCFFF792FB72
:10234000FFF774FBFFF7FAFBFFF7DEFB3E4B3F4A5C
:1023500018883F491080002801D0884201D101200F
:10236000108058883B4D7D22D2002880002801D063
:10237000884200D12A809888374E0028308001D0CA
:10238000884200D132803548FEF760FC3448FEF7C1
:10239000FAFF202233493248FFF73AFA0924E406CB
:1023A000002280212046FEF70FFC0022402120461B
:1023B000FEF70AFC2C4F2948FEF748FC00221021AA
:1023C0002046FEF701FC012280212046FEF7FCFB9F
:1023D000002208212046FEF7F7FB2888FEF78CFA3A
:1023E000002280212046FEF7EFFB01220821204633
:1023F000FEF7EAFB6420FEF77FFA01221021204657
:10240000FEF7E2FB012240212046FEF7DDFB012220
:1024100008212046FEF7D8FB3088FEF76DFA00222F
:1024200040212046FEF7D0FB002208212046FEF77F
:10243000CBFB6420FEF760FA38780028BBD0FFF7AA
:102440001FFF00203870B6E7003C0008060000209F
:10245000FFFF00000200002004000020B400002064
:10246000C4000020240000200000002070B50925D1
:102470000446ED06012220212846FEF7A5FB224650
:1024800007490848FFF7F8F90748FEF785F90128DA
:10249000FAD1002220212846FEF796FB70BD0000ED
:1024A00044000020C40000208C01002010B586B03C
:1024B0000020009001900290154C0120039404909C
:1024C000FEF7C4FA05A902A8FEF728FA002802D0F0
:1024D000012006B010BD0F496A46C8881070000A76
:1024E000507048889070000AD07088881071000A77
:1024F000507121460320019B009AFEF769FA0028DB
:1025000001D00320E5E7FEF759FA0020E1E70000DB
:10251000003C00080000002000C1814001C0804153
:1025200001C0804100C1814001C0804100C18140A3
:1025300000C1814001C0804101C0804100C1814093
:1025400000C1814001C0804100C1814001C0804183
:1025500001C0804100C1814001C0804100C1814073
:1025600000C1814001C0804100C1814001C0804163
:1025700001C0804100C1814000C1814001C0804153
:1025800001C0804100C1814001C0804100C1814043
:1025900000C1814001C0804101C0804100C1814033
:1025A00000C1814001C0804100C1814001C0804123
:1025B00001C0804100C1814000C1814001C0804113
:1025C00001C0804100C1814001C0804100C1814003
:1025D00000C1814001C0804100C1814001C08041F3
:1025E00001C0804100C1814001C0804100C18140E3
:1025F00000C1814001C0804101C0804100C18140D3
:1026000000C1814001C0804100C1814001C08041C2
:1026100001C0804100C1814000C0C101C30302C2AA
:10262000C60607C705C5C404CC0C0DCD0FCFCE0E12
:102630000ACACB0BC90908C8D81819D91BDBDA1A82
:102640001EDEDF1FDD1D1CDC14D4D515D71716D6F2
:10265000D21213D311D1D010F03031F133F3F23262
:1026600036F6F737F53534F43CFCFD3DFF3F3EFED2
:10267000FA3A3BFB39F9F83828E8E929EB2B2AEA42
:10268000EE2E2FEF2DEDEC2CE42425E527E7E626B2
:1026900022E2E323E12120E0A06061A163A3A26222
:1026A00066A6A767A56564A46CACAD6DAF6F6EAE92
:1026B000AA6A6BAB69A9A86878B8B979BB7B7ABA02
:1026C000BE7E7FBF7DBDBC7CB47475B577B7B67672
:1026D00072B2B373B17170B05090915193535292E2
:1026E00096565797559594549C5C5D9D5F9F9E5E52
:1026F0005A9A9B5B99595898884849894B8B8A4AC2
:102700004E8E8F4F8D4D4C8C448485458747468631
:1027100082424383418180400000000000000000AD
:102720000102030406070809000000000102030477
:10273000502700080000002024000000F4000008DA
:1027400074270008240000202C0800001001000855
:102750000000E803E80301000000000000000000A2
:102760000000000001000000040000000000000064
:0427700000127A00D9
:04000005080000B13E
:00000001FF
